:020000040000FA
:060000001C308A000C2CEC
:103800001C308A00022C8A01000000000000000029
:103810001C308A000A2CFF3F8316031307148312FF
:103820000313071C1B2C1D25E324831203178C088C
:10383000031D1B2C032CEF245C2583120313A5010D
:10384000A7019E2524241D2C292516250A3A031993
:10385000252C0A3A3A3A031D252C32240038031D40
:10386000242C0800A301FE241F39A2000310A20C7F
:10387000FE24A000FE24A1000310A00CA10C213006
:103880002006031D432CFE24013A0319672C260849
:10389000003A031D632CAB24FE242308031D6D2C6A
:1038A0002D25271C3F2583120313203020060319E2
:1038B000632C213020060319622C0310E43020070A
:1038C00003186F2C7124B8242E300E250134B8242F
:1038D0001D258E018C01C1240034A6250134B82594
:1038E00001342A3084002208A4002008031D862CFD
:1038F0002518862CFC3021070318862C2108043E4D
:10390000831203178D001C308F00932C2514831213
:1039100003132008831203178F0083120313210857
:10392000831203178D0000088C00840A00088E00A3
:10393000840A21308312031320060319A12CC12409
:10394000A22CCD2483120313A10FA82CA00A752C3E
:10395000A40B752C08002A3084002208A400FE2441
:103960008000840AFE248000840AA40BAF2C080087
:1039700016250A3A0319B82C0A3A0D3A0319080019
:10398000B82C8316031784308C0055308D00AA3074
:103990008D008C1400000000080000308312031713
:1039A0008F00831603178C18D32C04308C005530ED
:1039B0008D00AA308D008C14000000008C18DE2CC5
:1039C0008C1D00340134831203171F308F058316BA
:1039D000031780308C000C140000000008008312D4
:1039E000031306178316031306136730990018157F
:1039F0009816831203131816981708001625BF3E51
:103A0000031C073E0A3EA600A60E1625BF3E031C59
:103A1000073E0A3EA6042608A307080083120313E4
:103A2000861B102D0C1E122D990008008312031303
:103A300006138C1E192D1A080800831203171C3058
:103A40008F000B308D0008000D300E250A300E253A
:103A500008008312031306130800831203130617CA
:103A60000800A800280E37252808372508000F3938
:103A7000F63E0318073E0A3E303E0E25080083122C
:103A800003130130A7001D253F308E00FF308C004E
:103A9000C124831203134D2508004C300E256F30CE
:103AA0000E2561300E2564300E2569300E256E30EE
:103AB0000E2567300E250800242543300E256F3073
:103AC0000E256D300E2570300E2575300E256230B6
:103AD0000E256F300E2574300E2569300E256330AB
:103AE0000E2573300E2520300E2552300E25433022
:103AF0000E2534300E2530300E2520300E25423074
:103B00000E256F300E256F300E2574300E256C306B
:103B10000E256F300E2561300E2564300E25653080
:103B20000E2572300E2520300E2556300E253130F0
:103B30000E252E300E2534300E25080024254F305A
:103B40000E254B300E253E300E2508002425423030
:103B50000E2561300E2564300E2520300E254C30A8
:103B60000E2569300E256E300E2565300E250800B5
:103B7000242542300E2561300E2564300E2520307C
:103B80000E2561300E2564300E2564300E2572300E
:103B90000E2565300E2573300E2573300E25080076
:02400E00723FFF
:00000001FF
